:100000000C942A000C945F141895000018950000B9
:10001000189500001895000018950000189500002C
:10002000189500001895000018950000189500001C
:10003000189500001895000018950000189500000C
:1000400018950000189500001895000018950000FC
:10005000189500008FE58DBFC0E2E8E74E2E88E0DE
:100060008EBFD8E0F7E05F2EEEEFF7E0A0E6B0E05D
:1000700088278D933197E9F78FEC89B980E080BDAF
:1000800088E18AB90E94AC15662480E08ABB8FEFB4
:1000900087BB8A9882E085BF85E088BB84E082BB0D
:1000A00078948BB780648BBFC29A0E9491158CE0C4
:1000B0000E94FA1580E08093230380E08093680318
:1000C00080E090E0A8E3B4E08D939C9380E090E022
:1000D000AAE3B4E08D939C9381E08093D100A7E8DC
:1000E000B2E088278C93A4E9B2E088278C93A1EA38
:1000F000B2E088278C93AEEAB2E088278C93ABEB12
:10010000B2E088278C93A8ECB2E088278C93A5ED09
:10011000B2E088278C93A2EEB2E088278C93AFEEF2
:10012000B2E088278C93ACEFB2E088278C93A9E0EB
:10013000B3E088278C93A6E1B3E088278C93A7EDE2
:10014000B0E0ECE1FBE40E94DB217894A3E4B2E0B0
:10015000E8E7FAE40E946E1FABE4B2E0E0E8FAE4FC
:100160000E946E1F0027A9E3B0E08C9187FB0EF47C
:1001700001E041E0041711F00C94C0000C94F4006D
:100180000027A9E3B0E08C9186FB0EF401E041E08A
:10019000041711F00C94CE000C9421028FE711E0AB
:1001A0000E94A015EEE1FBE40E948A158FEB11E09E
:1001B0000E94A015E4E3FBE40E948A1583E911E0A4
:1001C0000E94A015EAE4FBE40E948A1583ED11E089
:1001D0000E94A015E0E6FBE40E948A15E3E0F0E04F
:1001E0000E94A3150C94D402C29A8FE711E00E94DA
:1001F000A015E6E7FBE40E948A158FEB11E00E9450
:10020000A015ECE8FBE40E948A1583E911E00E9446
:10021000A015E2EAFBE40E948A1583ED11E00E943A
:10022000A015E8EBFBE40E948A150E947B15EEEC1A
:10023000FBE40E9474150E947B150E947B15E4EE7E
:10024000FBE40E9474150E947B15ECE1FCE40E9423
:1002500074150E947B150E946815A0EDB0E08C9388
:10026000A0EDB0E08C91A8E6B0E08F930E946115FC
:100270008F918D9388278C9381E00E943616A0ED94
:10028000B0E08C91A881B9818D9388278C93A88147
:10029000B981EEE3FCE40E9428250FB681E0481AFC
:1002A0008827580A22960FBE11F40C945C01A0ED29
:1002B000B0E08C910E947E150091D000033211F0C5
:1002C0000C942B01E0E1F0E0A8E6B0E09DE07BE7D4
:1002D0000E940D250E947B15E0E4FCE40E94741549
:1002E000E0E1F0E0ACE9B0E09DE00E941B25ACE964
:1002F000B0E00E946E150E947B15ACE9B0E00E9450
:100300002225082F41E0041BABEDB0E00C93ECE993
:10031000F0E00091DB00ACE9B0E00E94FF248FEB3D
:1003200019E00E94A015ACE9B0E00E9484150E947B
:100330007B15E0E6FCE40E9474150E947B15E8E959
:10034000FCE40E9474150E947B150E946815A0EDC4
:10035000B0E08C93A0EDB0E08C91A5E7B0E08F9376
:100360000E9461158F918D9388278C9381E00E9464
:100370003616A0EDB0E08C91A881B9818D938827C5
:100380008C93A881B981EEE3FCE40E9428250FB686
:1003900081E0481A8827580A22960FBE11F40C945F
:1003A000D601A0EDB0E08C910E947E150091D000A6
:1003B000033211F00C94A501E0E2F0E0A5E7B0E013
:1003C0009DE07BE70E940D250E947B15E0E4FCE4A4
:1003D0000E947415E0E2F0E0A9EAB0E09DE00E941E
:1003E0001B25A9EAB0E00E946E150E947B15A9EAC0
:1003F000B0E00E942225082F41E0041BABEDB0E0E5
:100400000C93E9EAF0E00091DB00A9EAB0E00E9479
:10041000FF2483E919E00E94A015A9EAB0E00E9438
:1004200084150E947B15E8EBFCE40E9474150E9481
:100430007B15ECEDFCE40E9474150E947B15F8948A
:10044000FFCFC29A8FE711E00E94A015E6E7FBE418
:100450000E948A158FEB11E00E94A015E8EBFBE4E7
:100460000E948A1583E911E00E94A015E8EBFBE4E5
:100470000E948A1583ED11E00E94A015E4E1FDE4DD
:100480000E948A150E947B15EEECFBE40E94741515
:100490000E947B150E947B15EAE2FDE40E94741520
:1004A0000E947B15ECE1FCE40E9474150E947B1510
:1004B0000E946815A0EDB0E08C93A0EDB0E08C91A7
:1004C000A2E8B0E08F930E9461158F918D938827E9
:1004D0008C9381E00E943616A0EDB0E08C91A8814B
:1004E000B9818D9388278C93A881B981EEE3FCE4D0
:1004F0000E9428250FB681E0481A8827580A2296BC
:100500000FBE11F40C948902A0EDB0E08C910E9412
:100510007E150091D000033211F00C945802E0E3F4
:10052000F0E0A2E8B0E09DE07BE70E940D250E948C
:100530007B15E0E4FCE40E947415E0E3F0E0A6EB38
:10054000B0E09DE00E941B25A6EBB0E00E946E1576
:100550000E947B15A6EBB0E00E942225082F41E007
:10056000041BABEDB0E00C93E6EBF0E00091DB0098
:10057000A6EBB0E00E94FF2483ED19E00E94A015D5
:10058000A6EBB0E00E9484150E947B15E8EBFCE42A
:100590000E9474150E947B15ECEDFCE40E9474151A
:1005A0000E947B15F894FFCF8FE711E00E94A01501
:1005B000E6E5FDE40E948A158FEB11E00E94A0158C
:1005C000E8EBFBE40E948A1583E911E00E94A01584
:1005D000E8EBFBE40E948A1583ED11E00E94A01570
:1005E000E8EBFBE40E948A15E1E0F0E00E94A3152D
:1005F0000027A9E3B0E08C9183FB0EF401E041E019
:10060000041711F00C9406030C9479055A924A923F
:10061000A42DB52DECE6FDE40E94DB2187E00E94CD
:1006200020150E949914229687E00E941C15E8E28A
:10063000F3E0FA93EA930E94E9142296E5E3F3E0EB
:10064000FA93EA930E94E9142296E8E3F3E0FA931E
:10065000EA930E94E9142296E5E4F3E0FA93EA9320
:100660000E94E9142296E8E4F3E0FA93EA930E94E8
:10067000E914229691E09A93A8E4B3E0E4E7FDE45C
:100680002FEF0E94E121A2E5B4E00C93A2E5B4E0D3
:100690008C9181508C93E8E4F3E000915204A8E43B
:1006A000B3E00E94FF2481E0E8E2F3E002E00A9375
:1006B000A4E7B1E00E94F82483E0E8E2F3E002E07E
:1006C0000A93A7E7B1E00E94F82486E0E8E2F3E0AD
:1006D00002E00A93AAE7B1E00E94F824AAE7B1E099
:1006E0000E942225082F013011F00C947F03AAE705
:1006F000B1E00E946115E6E7FDE40E94DB2181E0A4
:10070000E8E3F3E003E00A93A7EAB1E00E94F824EB
:1007100084E0E8E3F3E002E00A93ABEAB1E00E9490
:10072000F82487E0E8E3F3E002E00A93AEEAB1E000
:100730000E94F824AEEAB1E00E942225082F013081
:1007400011F00C94AB03AEEAB1E00E946115E6E74C
:10075000FDE40E94DB21A5E3B3E0E8E7FDE40E94AD
:10076000282511F00C94BC03A1E8B2E0ECE1FBE415
:100770000E94DB210C94C003A1E8B2E088278C938F
:10078000A5E4B3E0EAE7FDE40E94282511F00C940B
:10079000D103A1E8B2E0ECE1FBE40E94DB210C9480
:1007A000D503A4E8B2E088278C93A4E7B1E00E94C7
:1007B0002A23EDE0F0E0ADE7B1E00E94F224A7E7E4
:1007C000B1E00E942A23EDE0F0E0A1E8B1E00E9450
:1007D000F224E8E8FAE40E940B23E1E8F1E00E9449
:1007E0001B220E945A22EDE0F0E0A1E8B1E00E9455
:1007F000F224AAE7B1E00E942A23EDE0F0E0A5E8A8
:10080000B1E00E94F224ECE8FAE40E940B23E5E850
:10081000F1E00E941B220E945A22EDE0F0E0A5E8E0
:10082000B1E00E94F224EDE7F1E00E942022E5E829
:10083000F1E00E941B220E94B922EDE0F0E0A5E861
:10084000B1E00E94F224E1E8F1E00E942022E5E814
:10085000F1E00E941B220E94B922EDE0F0E0A5E841
:10086000B1E00E94F224A9E8B1E0E5E8F1E00E94DD
:100870001B220E943C168EE00E943616E9E8F1E049
:10088000A881B9810E94ED24E1E8F2E0A9E8B1E095
:100890000E94ED24E881F981A9E8B1E00E94611588
:1008A0000E94ED248EE0481A8827580A2296A9E86B
:1008B000B1E00E942A23EDE0F0E0A3EAB1E00E945B
:1008C000F224A7EAB1E00E942A23EDE0F0E0A1EBD8
:1008D000B1E00E94F224ABEAB1E00E942A23EDE0ED
:1008E000F0E0A5EBB1E00E94F224E8E8FAE40E940F
:1008F0000B23E5EBF1E00E941B220E945A22EDE05F
:10090000F0E0A5EBB1E00E94F224AEEAB1E00E9473
:100910002A23EDE0F0E0A9EBB1E00E94F224ECE83C
:10092000FAE40E940B23E9EBF1E00E941B220E94F3
:100930005A22EDE0F0E0A9EBB1E00E94F224E1EBF5
:10094000F1E00E942022E9EBF1E00E941B220E94CC
:10095000B922EDE0F0E0A9EBB1E00E94F224E5EB72
:10096000F1E00E942022E9EBF1E00E941B220E94AC
:10097000B922EDE0F0E0A9EBB1E00E94F224ADEB8A
:10098000B1E0E9EBF1E00E941B220E943C168EE0F0
:100990000E943616EDEBF1E0A881B9810E94ED24AA
:1009A000E4E8F2E0ADEBB1E00E94ED24E881F981EA
:1009B000ADEBB1E00E9461150E94ED248EE0481A73
:1009C0008827580A2296ADEBB1E00E942A23EDE079
:1009D000F0E0A7EDB1E00E94F224E5E3F3E001E0EE
:1009E000A8EEB3E00E94FF24E5E4F3E001E0ABEE03
:1009F000B3E00E94FF24E4E7F1E0AEECB3E00E9434
:100A0000ED24AEECB3E00E946115ECE7FDE40E943A
:100A1000DB21E7E7F1E0AEECB3E00E9461150E9454
:100A2000ED24AEECB3E00E946115EEE7FDE40E9418
:100A3000DB21EAE7F1E0AEECB3E00E9461150E9431
:100A4000ED24E8EEF3E0AEECB3E00E9461150E9405
:100A5000ED24E7EAF1E0ABEDB3E00E94ED24ABED6D
:100A6000B3E00E946115ECE7FDE40E94DB21EBEAB4
:100A7000F1E0ABEDB3E00E9461150E94ED24ABED17
:100A8000B3E00E946115EEE7FDE40E94DB21EEEA8F
:100A9000F1E0ABEDB3E00E9461150E94ED24EBEEB6
:100AA000F3E0ABEDB3E00E9461150E94ED24EEECA3
:100AB000F3E0A4EAB3E00E94ED24A4EAB3E00E94CC
:100AC0006115E0E8FDE40E94DB21EBEDF3E0A4EA30
:100AD000B3E00E9461150E94ED24E3EAF1E0ABEE81
:100AE000B1E00E94F620E7EDF1E0A3EFB1E00E9453
:100AF000F6200027A9E3B0E08C9180FB0EF401E022
:100B000040E0041711F00C9487050C94CB078091FA
:100B1000D90080688093D900C2988FEC89B95A9225
:100B20004A92A42DB52DE2E8FDE40E94DB2188E085
:100B30000E9420150E949914229688E00E941C159C
:100B4000EBE5F2E0FA93EA930E94E9142296EDE5D0
:100B5000F2E0FA93EA930E94E9142296EFE5F2E0BC
:100B6000FA93EA930E94E9142296AFE5B2E00E945C
:100B70002225082F41E0041BABEDB0E00C93EFE51C
:100B8000F2E00091DB00AFE5B2E00E94FF24EBE76A
:100B9000F2E0FA93EA930E94E9142296ABE7B2E0FE
:100BA0000E942225082F41E0041BABEDB0E00C931E
:100BB000EBE7F2E00091DB00ABE7B2E00E94FF243C
:100BC000EAE6F2E0FA93EA930E94E9142296AAE692
:100BD000B2E00E942225082F41E0041BABEDB0E0FB
:100BE0000C93EAE6F2E00091DB00AAE6B2E00E9494
:100BF000FF24EEE7F2E0FA93EA930E94E9142296CA
:100C0000AEE7B2E00E942225082F41E0041BABEDC5
:100C1000B0E00C93EEE7F2E00091DB00AEE7B2E06B
:100C20000E94FF24ABE7B2E0E8E7FDE40E9428253C
:100C300011F00C942306ABE7B2E0ECE1FBE40E9478
:100C4000DB210C942706ABE7B2E088278C93AEE754
:100C5000B2E0EAE7FDE40E94282511F00C94380682
:100C6000AEE7B2E0ECE1FBE40E94DB210C943C0631
:100C7000AEE7B2E088278C9381E0EFE5F2E002E096
:100C80000A93ACEDB0E00E94F82483E0EFE5F2E0D7
:100C900002E00A93A0EEB0E00E94F82486E0EFE5BF
:100CA000F2E003E00A93A4EEB0E00E94F824A4EE80
:100CB000B0E00E942225082F023011F00C94680643
:100CC000A4EEB0E00E946115E6E7FDE40E94DB219E
:100CD000A4EEB0E00E942225082F013011F00C9400
:100CE0007906A4EEB0E00E946115EAE8FDE40E94F6
:100CF000DB21ACEDB0E00E942A23EDE0F0E0A7E0BC
:100D0000B1E00E94F224A0EEB0E00E942A23EDE0C0
:100D1000F0E0ABE0B1E00E94F224E8E8FAE40E94DF
:100D20000B23EBE0F1E00E941B220E945A22EDE02F
:100D3000F0E0ABE0B1E00E94F224A4EEB0E00E944B
:100D40002A23EDE0F0E0AFE0B1E00E94F224E0E918
:100D5000FAE40E940B23EFE0F1E00E941B220E94C4
:100D60005A22EDE0F0E0AFE0B1E00E94F224EBE0C7
:100D7000F1E00E942022E7E0F1E00E941B220E94A5
:100D8000B922EDE0F0E0A3E1B1E00E94F224E3E15A
:100D9000F1E00E942022EFE0F1E00E941B220E947D
:100DA000B922EDE0F0E0A3E1B1E00E94F224A7E176
:100DB000B1E0E3E1F1E00E941B220E943C168EE0CC
:100DC0000E943616E7E1F1E0A881B9810E94ED2486
:100DD000EBE7F2E0A7E1B1E00E94ED24E881F981C0
:100DE000A7E1B1E00E9461150E94ED248EE0481A4F
:100DF0008827580A2296A7E1B1E0EBEDF1E00E94C6
:100E00004C1E81E0EAE6F2E003E00A93A0EFB0E0D6
:100E10000E94F82484E0EAE6F2E002E00A93A4EFFC
:100E2000B0E00E94F82487E0EAE6F2E003E00A93EB
:100E3000A8EFB0E00E94F824A8EFB0E00E942225BD
:100E4000082F023011F00C942D07A8EFB0E00E949B
:100E50006115E6E7FDE40E94DB21A8EFB0E00E9407
:100E60002225082F013011F00C943E07A8EFB0E0C6
:100E70000E946115EAE8FDE40E94DB21A0EFB0E0EA
:100E80000E942A23EDE0F0E0AFE3B1E00E94F224FB
:100E9000A4EFB0E00E942A23EDE0F0E0A3E4B1E08B
:100EA0000E94F224E8E8FAE40E940B23E3E4F1E074
:100EB0000E941B220E945A22EDE0F0E0A3E4B1E080
:100EC0000E94F224A8EFB0E00E942A23EDE0F0E0B7
:100ED000A7E4B1E00E94F224E0E9FAE40E940B23C7
:100EE000E7E4F1E00E941B220E945A22EDE0F0E0CC
:100EF000A7E4B1E00E94F224E3E4F1E00E942022A2
:100F0000EFE3F1E00E941B220E94B922EDE0F0E045
:100F1000ABE4B1E00E94F224EBE4F1E00E94202275
:100F2000E7E4F1E00E941B220E94B922EDE0F0E02C
:100F3000ABE4B1E00E94F224AFE4B1E0EBE4F1E015
:100F40000E941B220E943C168EE00E943616EFE49F
:100F5000F1E0A881B9810E94ED24EEE7F2E0AFE470
:100F6000B1E00E94ED24E881F981AFE4B1E00E9494
:100F700061150E94ED248EE0481A8827580A2296AF
:100F8000AFE4B1E0E3EEF1E00E944C1EC29A8FECB8
:100F900089B90C940E088091D9008F778093D9007D
:100FA000E0E1F0E0ACE9B0E09DE00E941B25ACE997
:100FB000B0E00E942225082F41E0041BABEDB0E019
:100FC0000C93ECE9F0E00091DB00ACE9B0E00E94AA
:100FD000FF24ACE9B0E0EBEDF1E00E944C1EE0E252
:100FE000F0E0A9EAB0E09DE00E941B25A9EAB0E08C
:100FF0000E942225082F41E0041BABEDB0E00C93CA
:10100000E9EAF0E00091DB00A9EAB0E00E94FF24E9
:10101000A9EAB0E0E3EEF1E00E944C1EEBEDF1E056
:10102000ABEFB1E00E940B1AEBEFF1E0ABEFB1E0F8
:101030000E94EA17EBEEF1E0A3E0B2E00E940B1A87
:10104000E3E0F2E0A3E0B2E00E94EA17EBEDF1E0AA
:10105000ABE0B2E00E940B1AEBE0F2E0ABE0B2E0F2
:101060000E94E617EBEEF1E0A3E1B2E00E940B1A5A
:10107000E3E1F2E0A3E1B2E00E94E617ABE1B2E007
:10108000BA93AA93A3EFB1E0E3EEF1E00E94771BDD
:101090002296EBE1F2E0ABE1B2E00E940B1AEBE149
:1010A000F2E0ABE1B2E00E94E617A3E2B2E0BA934D
:1010B000AA93A3E0B2E0EBEFF1E00E94C71B2296F7
:1010C000ABE2B2E0BA93AA93A3E1B2E0EBE0F2E0C4
:1010D0000E94C71B2296ABE2B2E0BA93AA93ABE19F
:1010E000B2E0EBE2F2E00E94C71B2296ABE2B2E074
:1010F000BA93AA93A3E2B2E0EBE2F2E00E948C1B67
:101100002296EBE2F2E0ABE2B2E00E94D8180027B0
:10111000A9E3B0E08C9185FB0EF401E041E00417F7
:1011200011F00C9495080C94B608ABE3B2E0BA93B6
:10113000AA93E4E9FAE4A0E6B0E00E946E1FEBE2B5
:10114000F2E00E94C71B2296A8E0B4E0EBE3F2E0D5
:101150000027A8E0B4E00E94D61CE8E0F4E005E037
:10116000A8E0B4E00E94FF240C94D508ABE3B2E001
:10117000BA93AA93ECE9FAE4A0E6B0E00E946E1FED
:10118000EBE2F2E00E94C71B2296A8E0B4E0EBE39A
:10119000F2E00027A8E0B4E00E94D61CE8E0F4E00A
:1011A00005E0A8E0B4E00E94FF24ABEFB1E0BA9301
:1011B000AA93ABE4B2E0EBEDF1E00E94C71B2296EC
:1011C000A3E0B2E0BA93AA93ABE4B2E0E3EEF1E0BD
:1011D0000E94C71B2296ABE0B2E0BA93AA93ABE49D
:1011E000B2E0EBEEF1E00E94C71B2296A3E1B2E071
:1011F000BA93AA93ABE4B2E0E3EFF1E00E94C71B1D
:101200002296A3E5B2E0BA93AA93A3E1B2E0E3E0A9
:10121000F2E00E94771B2296EBEFF1E0ABE1B2E047
:101220000E94E617E3E5F2E0A3E2B2E00E94E617CF
:10123000EBE0F2E0ABE2B2E00E94E617A3E2B2E03C
:10124000BA93AA93A3E2B2E0EBE1F2E00E94C71BDB
:101250002296ABE2B2E0BA93AA93ABE2B2E0E3E249
:10126000F2E00E94C71B2296EBEFF1E0ABE1B2E0A7
:101270000E94EA17EBE0F2E0A3E2B2E00E94EA1774
:10128000A3E2B2E0BA93AA93A3E2B2E0EBE1F2E008
:101290000E94C71B2296A3E3B2E0BA93AA93ABE2E3
:1012A000B2E0E3E2F2E00E948C1B2296ABE1B2E0F6
:1012B000BA93AA93A3E3B2E0E3E3F2E00E94C71B70
:1012C0002296ABE1B2E0BA93AA93E4EAFAE4A0E68C
:1012D000B0E00E946E1FE0E6F0E0ABE1B2E00E94F9
:1012E000771B2296EBE1F2E0ABE1B2E00E94B51988
:1012F000A3E3B2E0BA93AA93ABE1B2E0E3E3F2E096
:101300000E94261C2296E3E3F2E0A3E3B2E00E94EF
:101310002F19ABE1B2E0BA93AA93ECEAFAE4A0E6A3
:10132000B0E00E946E1FE3E4F2E00E94261C2296C9
:10133000A3E3B2E0BA93AA93A3E3B2E0EBE1F2E055
:101340000E94771B2296EBE0F2E0A3E1B2E00E945C
:10135000EA17EBEFF1E0ABE1B2E00E94EA17E3E35A
:10136000F2E0A3E2B2E00E94E617A3E2B2E0BA9391
:10137000AA93ABE1B2E0E3E2F2E00E94C71B22963F
:10138000A3E1B2E0BA93AA93A3E2B2E0E3E1F2E010
:101390000E94771B2296EBEFF1E0ABE1B2E00E94F6
:1013A000E617E3E3F2E0A3E2B2E00E94EA17ABE162
:1013B000B2E0BA93AA93A3E2B2E0EBE1F2E00E94BA
:1013C000C71B2296ABE2B2E0BA93AA93ABE1B2E0BC
:1013D000E3E1F2E00E94261C2296A3E1B2E0BA9378
:1013E000AA93ABE2B2E0EBE2F2E00E94C71B2296C6
:1013F000A3E1B2E0BA93AA93E4EAFAE4A0E6B0E08B
:101400000E946E1FE0E6F0E0A3E1B2E00E94771BCD
:101410002296E3E1F2E0A3E1B2E00E94B519ABE26B
:10142000B2E0BA93AA93A3E1B2E0EBE2F2E00E9449
:10143000261C2296EBE2F2E0ABE2B2E00E942F190A
:10144000A3E1B2E0BA93AA93ECEAFAE4A0E6B0E032
:101450000E946E1FE3E4F2E00E94261C2296ABE29B
:10146000B2E0BA93AA93ABE2B2E0E3E1F2E00E9409
:10147000771B2296ABE2B2E0BA93AA93ABE4B2E058
:10148000EBE2F2E00E94261C2296E3E5F2E0A3E5FF
:10149000B2E00E94EA17A3E5B2E0E4EBFAE40E94AE
:1014A000471F10F40C94650AABE2B2E0BA93AA931A
:1014B000ECEBFAE4A0E6B0E00E946E1FE0E6F0E09C
:1014C000ABE2B2E00E94771B2296ABE2B2E0E4EA24
:1014D000FAE40E94471F10F00C94740AABE2B2E0E9
:1014E000E4EBFAE40E946E1FABE2B2E0E4ECFAE453
:1014F0000E94471F80E010F009F081E08F93ABE27B
:10150000B2E0ECECFAE40E94471F81E008F080E0D2
:101510009F918923882311F40C94940AABE2B2E0E2
:10152000E4EDFAE40E946E1FABE2B2E0ECEDFAE407
:101530000E94471F80E010F009F081E08F93ABE23A
:10154000B2E0E4EEFAE40E94471F81E008F080E098
:101550009F918923882311F40C94B40AABE2B2E082
:10156000ECEEFAE40E946E1FABE2B2E0E4EFFAE4C4
:101570000E94471F80E010F009F081E08F93ABE2FA
:10158000B2E0ECEFFAE40E94471F81E008F080E04F
:101590009F918923882311F40C94D40AABE2B2E022
:1015A000E4E0FBE40E946E1FABE2B2E0ECE0FBE49F
:1015B0000E94471F18F011F00C94E00A0C94E60A00
:1015C000ABE2B2E0E4EBFAE40E946E1FAEEEB3E0F1
:1015D000EBE3F2E00027AEEEB3E00E94D61CAEEEE5
:1015E000B3E00E942A23EDE0F0E0A9EFB3E00E940F
:1015F000F224E9EFF3E00E941B22E4E1FBE40E9405
:101600000B230E94142310F00C94090B80E08093AC
:101610005404E9EFF3E00E941B22E4E1FBE40E94A2
:101620000B230E94142381E008F480E08F93E9EFFC
:10163000F3E00E941B22E8E1FBE40E940B230E94DE
:10164000142381E008F080E09F918923882311F41E
:101650000C942D0B81E080935404E9EFF3E00E9499
:101660001B22E8E1FBE40E940B230E94142310F4E8
:101670000C943D0B82E0809354040091540400309C
:1016800011F00C94590BA0E6B7E0AF93BF93E9EFCC
:10169000F3E00E941B220E943C1611E002E0BF9181
:1016A000AF910E940724E0E6F7E0ADEFB3E00E94BF
:1016B000ED2400915404013011F00C94750BA0E658
:1016C000B7E0AF93BF93E9EFF3E00E941B220E94C3
:1016D0003C1611E001E0BF91AF910E940724E0E6C3
:1016E000F7E0ADEFB3E00E94ED2400915404023026
:1016F00011F00C94910BA0E6B7E0AF93BF93E9EF24
:10170000F3E00E941B220E943C1611E000E0BF9112
:10171000AF910E940724E0E6F7E0ADEFB3E00E944E
:10172000ED24ADEFB3E00E942225A3E5B4E08C9355
:10173000A3E5B4E08C9181508C9300915404023065
:1017400011F00C94AB0BEDEFF3E000915304ADEF0F
:10175000B3E00E94FF240027A9E3B0E08C9184FB52
:101760000EF401E041E0041711F00C94B90B0C9455
:10177000C90BADEFB3E00E946115EEE8FDE40E94F5
:10178000DB21A4E7B3E0E0E9FDE40E94DB210C9457
:10179000D70BADEFB3E00E946115E2E9FDE40E94D2
:1017A000DB21A4E7B3E0E4E9FDE40E94DB21EBE206
:1017B000F2E0A0E6B0E00E949C1CA2E2B4E0E0E609
:1017C000F0E00027A2E2B4E00E94D61CE2E2F4E0DE
:1017D000ADE2B4E00E94ED24ADE2B4E00E946115F8
:1017E000ECE7FDE40E94DB210E9491150027A9E3AC
:1017F000B0E08C9181FB0EF401E041E0041711F0A0
:101800000C94040C0C94C7110027A9E3B0E08C9150
:1018100082FB0EF401E041E0041711F00C94120C6D
:101820000C9477110027A9E3B0E08C9183FB0EF4B0
:1018300001E041E0041711F00C94200C0C94BB1053
:10184000E8E5F3E0A8E4B3E00E942A2511F00C9447
:101850002B0C0C94360CA3E2B3E08C918F5F8C932D
:10186000E8E4F3E0A8E5B3E00E94ED24009123034F
:10187000053011F00C943F0C81E08093230300911C
:101880002303013011F00C944B0CE8E4F3E0A7E8DB
:10189000B2E00E94ED2400912303023011F00C9479
:1018A000570CE8E4F3E0A4E9B2E00E94ED240091D3
:1018B0002303033011F00C94630CE8E4F3E0A1EA95
:1018C000B2E00E94ED2400912303043011F00C9447
:1018D0006F0CE8E4F3E0AEEAB2E00E94ED24009180
:1018E0002303013011F00C947B0CEDEFF3E0ABEB34
:1018F000B2E00E94ED2400912303023011F00C9419
:10190000870CEDEFF3E0A8ECB2E00E94ED2400912B
:101910002303033011F00C94930CEDEFF3E0A5EDED
:10192000B2E00E94ED2400912303043011F00C94E6
:101930009F0CEDEFF3E0A2EEB2E00E94ED240091E7
:101940002303013011F00C94AB0CEDE2F4E0AFEEA8
:10195000B2E00E94ED2400912303023011F00C94B8
:10196000B70CEDE2F4E0ACEFB2E00E94ED240091A0
:101970002303033011F00C94C30CEDE2F4E0A9E072
:10198000B3E00E94ED2400912303043011F00C9485
:10199000CF0CEDE2F4E0A6E1B3E00E94ED2400916B
:1019A0002303013011F00C94D90C83ED11E00E9457
:1019B000A01500912303013011F00C94E30CA7E86B
:1019C000B2E00E94841500912303013011F00C94C1
:1019D000ED0C83ED1BE00E94A01500912303013064
:1019E00011F00C94F70CABEBB2E00E94841500915F
:1019F0002303013011F00C94010D83ED11E10E94DD
:101A0000A01500912303013011F00C940B0DAFEEE3
:101A1000B2E00E94841500912303013011F00C9470
:101A2000150D8FE711E00E94A015009123030130EE
:101A300011F00C941F0DA4E9B2E00E9484150091EE
:101A40002303013011F00C94290D8FE71BE00E9455
:101A5000A01500912303013011F00C94330DA8EC74
:101A6000B2E00E94841500912303013011F00C9420
:101A70003D0D8FE711E10E94A01500912303013075
:101A800011F00C94470DACEFB2E00E948415009168
:101A90002303013011F00C94510D8FEB11E00E94E3
:101AA000A01500912303013011F00C945B0DA1EA05
:101AB000B2E00E94841500912303013011F00C94D0
:101AC000650D8FEB1BE00E94A015009123030130F0
:101AD00011F00C946F0DA5EDB2E00E9484150091F9
:101AE0002303013011F00C94790D8FEB11E10E946A
:101AF000A01500912303013011F00C94830DA9E08F
:101B0000B3E00E94841500912303013011F00C947E
:101B10008D0D83E911E00E94A0150091230301308F
:101B200011F00C94970DAEEAB2E00E94841500917A
:101B30002303013011F00C94A10D83E91BE00E94F6
:101B4000A01500912303013011F00C94AB0DA2EE0F
:101B5000B2E00E94841500912303013011F00C942F
:101B6000B50D83E911E10E94A01500912303013016
:101B700011F00C94BF0DA6E1B3E00E948415009112
:101B80002303023011F00C94C90D83E911E00E9487
:101B9000A01500912303023011F00C94D30DA7E897
:101BA000B2E00E94841500912303023011F00C94DE
:101BB000DD0D83E91BE00E94A01500912303023094
:101BC00011F00C94E70DABEBB2E00E94841500918C
:101BD0002303023011F00C94F10D83E911E10E940E
:101BE000A01500912303023011F00C94FB0DAFEE11
:101BF000B2E00E94841500912303023011F00C948E
:101C0000050E83ED11E00E94A01500912303023020
:101C100011F00C940F0EA4E9B2E00E94841500911B
:101C20002303023011F00C94190E83ED1BE00E9487
:101C3000A01500912303023011F00C94230EA8ECA0
:101C4000B2E00E94841500912303023011F00C943D
:101C50002D0E83ED11E10E94A015009123030230A7
:101C600011F00C94370EACEFB2E00E948415009195
:101C70002303023011F00C94410E8FE711E00E9413
:101C8000A01500912303023011F00C944B0EA1EA31
:101C9000B2E00E94841500912303023011F00C94ED
:101CA000550E8FE71BE00E94A01500912303023020
:101CB00011F00C945F0EA5EDB2E00E948415009126
:101CC0002303023011F00C94690E8FE711E10E949A
:101CD000A01500912303023011F00C94730EA9E0BB
:101CE000B3E00E94841500912303023011F00C949C
:101CF0007D0E8FEB11E00E94A015009123030230AE
:101D000011F00C94870EAEEAB2E00E9484150091A7
:101D10002303023011F00C94910E8FEB1BE00E9414
:101D2000A01500912303023011F00C949B0EA2EE3B
:101D3000B2E00E94841500912303023011F00C944C
:101D4000A50E8FEB11E10E94A01500912303023034
:101D500011F00C94AF0EA6E1B3E00E94841500913F
:101D60002303033011F00C94B90E8FEB11E00E94A5
:101D7000A01500912303033011F00C94C30EA7E8C3
:101D8000B2E00E94841500912303033011F00C94FB
:101D9000CD0E8FEB1BE00E94A015009123030330B2
:101DA00011F00C94D70EABEBB2E00E9484150091B9
:101DB0002303033011F00C94E10E8FEB11E10E942C
:101DC000A01500912303033011F00C94EB0EAFEE3D
:101DD000B2E00E94841500912303033011F00C94AB
:101DE000F50E83E911E00E94A01500912303033052
:101DF00011F00C94FF0EA4E9B2E00E94841500914A
:101E00002303033011F00C94090F83E91BE00E94B7
:101E1000A01500912303033011F00C94130FA8ECCC
:101E2000B2E00E94841500912303033011F00C945A
:101E30001D0F83E911E10E94A015009123030330D7
:101E400011F00C94270FACEFB2E00E9484150091C2
:101E50002303033011F00C94310F83ED11E00E9445
:101E6000A01500912303033011F00C943B0FA1EA5D
:101E7000B2E00E94841500912303033011F00C940A
:101E8000450F83ED1BE00E94A01500912303033052
:101E900011F00C944F0FA5EDB2E00E948415009153
:101EA0002303033011F00C94590F83ED11E10E94CC
:101EB000A01500912303033011F00C94630FA9E0E7
:101EC000B3E00E94841500912303033011F00C94B9
:101ED0006D0F8FE711E00E94A015009123030330DE
:101EE00011F00C94770FAEEAB2E00E9484150091D5
:101EF0002303033011F00C94810F8FE71BE00E9445
:101F0000A01500912303033011F00C948B0FA2EE67
:101F1000B2E00E94841500912303033011F00C9469
:101F2000950F8FE711E10E94A01500912303033064
:101F300011F00C949F0FA6E1B3E00E94841500916C
:101F40002303043011F00C94A90F8FE711E00E94D5
:101F5000A01500912303043011F00C94B30FA7E8EF
:101F6000B2E00E94841500912303043011F00C9418
:101F7000BD0F8FE71BE00E94A015009123030430E2
:101F800011F00C94C70FABEBB2E00E9484150091E6
:101F90002303043011F00C94D10F8FE711E10E945C
:101FA000A01500912303043011F00C94DB0FAFEE69
:101FB000B2E00E94841500912303043011F00C94C8
:101FC000E50F8FEB11E00E94A01500912303043070
:101FD00011F00C94EF0FA4E9B2E00E948415009177
:101FE0002303043011F00C94F90F8FEB1BE00E94D7
:101FF000A01500912303043011F00C940310A8ECF9
:10200000B2E00E94841500912303043011F00C9477
:102010000D108FEB11E10E94A015009123030430F5
:1020200011F00C941710ACEFB2E00E9484150091EF
:102030002303043011F00C94211083E911E00E9475
:10204000A01500912303043011F00C942B10A1EA89
:10205000B2E00E94841500912303043011F00C9427
:10206000351083E91BE00E94A01500912303043082
:1020700011F00C943F10A5EDB2E00E948415009180
:102080002303043011F00C94491083E911E10E94FC
:10209000A01500912303043011F00C945310A9E013
:1020A000B3E00E94841500912303043011F00C94D6
:1020B0005D1083ED11E00E94A01500912303043010
:1020C00011F00C946710AEEAB2E00E948415009102
:1020D0002303043011F00C94711083ED1BE00E9477
:1020E000A01500912303043011F00C947B10A2EE94
:1020F000B2E00E94841500912303043011F00C9487
:10210000851083ED11E10E94A01500912303043096
:1021100011F00C948F10A6E1B3E00E948415E6E95B
:10212000FDE40E947415A8E4B3E00E946E15EEE988
:10213000FDE40E947415A4E7B3E00E946E15EEE979
:10214000FDE40E947415A8E0B4E00E946E15E0EA78
:10215000FDE40E947415A2E2B4E00E946E150E9494
:102160007B15C098C19A84EF91E00E942716C09A0F
:10217000C1980C941814ABE7B2E0ECE1FBE40E94C8
:10218000282511F00C94CC10A6E8B3E0EAE7FDE4B2
:102190000E94DB210C94D210A6E8B3E0E4EAFDE44F
:1021A0000E94DB21AEE7B2E0ECE1FBE40E942825CF
:1021B00011F00C94E310A8E8B3E0E8E7FDE40E9416
:1021C000DB210C94E910A8E8B3E0E6EAFDE40E9404
:1021D000DB21AAE8B3E0EBEDF1E00027AAE8B3E0E9
:1021E0000E94D61CA7E9B3E0E3EEF1E00027A7E9DF
:1021F000B3E00E94D61CEAE8F3E008E0AAE8B3E006
:102200000E94FF24E7E9F3E008E0A7E9B3E00E94B9
:10221000FF248FE711E00E94A0150027A9EDB0E090
:102220008C9187FB0EF401E040E0041711F00C9450
:102230001D11E8EAFDE40E948A150027A9EDB0E02F
:102240008C9187FB0EF401E041E0041711F00C942F
:102250002D11E6EBFDE40E948A158FEB11E00E9440
:10226000A015E8ECFDE40E948A15AAE8B3E00E94FC
:10227000841583E911E00E94A015E2EDFDE40E94BF
:102280008A15A7E9B3E00E94841583ED11E00E944E
:10229000A0150027A9EDB0E08C9187FB0EF401E0BA
:1022A00040E0041711F00C945D11ECEDFDE40E9488
:1022B0008A15A9E6B3E00E9484150027A9EDB0E0D5
:1022C0008C9187FB0EF401E040E0041711F00C94B0
:1022D0006D11E1E0F0E00E94A315C098C19A84EF6F
:1022E00091E00E942716C09AC1980C9418148FE7A9
:1022F00011E00E94A015E6EEFDE40E948A158FEB26
:1023000011E00E94A015E4EFFDE40E948A15A8E404
:10231000B3E00E94841583E911E00E94A015ECEF60
:10232000FDE40E948A1583ED11E00E94A015A4EA45
:10233000B3E00E948415E6E9FDE40E947415A8E468
:10234000B3E00E946E15EEE9FDE40E947415A4E767
:10235000B3E00E946E15EEE9FDE40E947415A8E05A
:10236000B4E00E946E15E0EAFDE40E947415A2E25A
:10237000B4E00E946E150E947B15C098C19A84EF4C
:1023800091E00E942716C09AC1980C9418140091ED
:10239000D100003011F00C94D01180E080936803DC
:1023A0000091D100003011F00C94DC1180E090E03D
:1023B000A8E3B4E08D939C930091D100003011F01C
:1023C0000C94E81180E090E0AAE3B4E08D939C9334
:1023D0000091D100003011F00C94F211ACE3B4E0A4
:1023E00088278C930091D100003011F00C94FC11DF
:1023F000A7E4B4E088278C930091D100003011F05D
:102400000C940612A9EBB3E088278C930091D100BD
:10241000003011F00C941A12E7E7F3E0AFE8B0E0F7
:102420000E94ED24AFE8B0E00E946115E0E8FDE411
:102430000E94DB210091D100003011F00C94281291
:10244000E0E4F0E0AFE8B0E09DE07BE70E940D251E
:1024500081E08093D100E8E4F3E0A7E7B3E00E94D5
:10246000ED240027A9E3B0E08C9185FB0EF401E098
:1024700041E0041711F00C943F120C945A12E0E45E
:10248000F0E0A3ECB0E09DE00E941B25A3ECB0E0DF
:102490000E942225082F41E0041BABEDB0E00C9315
:1024A000E3ECF0E00091DB00A9E6B3E00E94FF243A
:1024B0000C947312E0E3F0E0A6EBB0E09DE00E9424
:1024C0001B25A6EBB0E00E942225082F41E0041B4B
:1024D000ABEDB0E00C93E6EBF0E00091DB00A9E699
:1024E000B3E00E94FF248FE711E00E94A015E6E010
:1024F000FEE40E948A15A8E4B3E00E9484158FEBE5
:1025000011E00E94A015E9E6F3E009E0A9E6B3E0D6
:102510000E94FF24ECEDFDE40E948A15A9E6B3E0D9
:102520000E948415E8E4F3E0A9E6B3E00E942A25BE
:1025300011F40C949D120C946E13E6E9FDE40E94D4
:102540007415A8E4B3E00E946E15EEE9FDE40E9464
:102550007415A4E7B3E00E946E15EEE9FDE40E9455
:102560007415A8E0B4E00E946E15E0EAFDE40E9454
:102570007415A2E2B4E00E946E150E947B1581E002
:1025800080936803A8E3B4E00D911C9141E050E012
:10259000040F151FA8E3B4E00D931C93A8E3B4E067
:1025A0000D911C91083E53E0150711F00C94DE12BA
:1025B00081E090E0A8E3B4E08D939C9383E911E07F
:1025C0000E94A015E0E1FEE40E948A15ADEFB3E0A1
:1025D0000E948415E4E1FEE40E948A15ADE2B4E0B5
:1025E0000E94841583E912E10E94A015A2E8B3E0DD
:1025F000E8E3F4E00E946224A2E8B3E00E9422250E
:10260000082F013011F00C94211385E00E9436163A
:10261000E2E8F3E0A881B9810E94ED24A2E8B3E0EA
:10262000EAE8FDE40E94DB21E881F981A2E8B3E059
:102630000E9461150E94ED2485E0481A8827580AF7
:102640002296A2E8B3E00E942225082F023011F062
:102650000C94461385E00E943616E2E8F3E0A88168
:10266000B9810E94ED24A2E8B3E0E6E7FDE40E9410
:10267000DB21E881F981A2E8B3E00E9461150E94A4
:10268000ED2485E0481A8827580A2296A2E8B3E08C
:102690000E94841583ED11E00E94A015A4EAB3E026
:1026A0000E948415EDEFF3E0ACE3B4E00E94ED246A
:1026B000EDE2F4E0A7E4B4E00E94ED24A8E3B4E086
:1026C0008D919C91AAE3B4E08D939C93E4EAF3E0AE
:1026D000A9EBB3E00E94ED240C9410148FEB14E1ED
:1026E0000E94A01500916803013011F00C947C1336
:1026F000E4E7FDE40E948A1583E911E00E94A01539
:1027000000916803003011F00C948A13E8EBFBE4AD
:102710000E948A1500916803013011F00C94A013F7
:10272000E0E1FEE40E948A15ACE3B4E00E94841567
:10273000E4E1FEE40E948A15A7E4B4E00E94841557
:1027400083E912E10E94A015A2E8B3E0EAE3F4E015
:102750000E946224A2E8B3E00E942225082F0130E3
:1027600011F00C94CF1385E00E943616E2E8F3E0F6
:10277000A881B9810E94ED24A2E8B3E0EAE8FDE473
:102780000E94DB21E881F981A2E8B3E00E94611593
:102790000E94ED2485E0481A8827580A2296A2E86C
:1027A000B3E00E942225082F023011F00C94F4139C
:1027B00085E00E943616E2E8F3E0A881B9810E9424
:1027C000ED24A2E8B3E0E6E7FDE40E94DB21E88126
:1027D000F981A2E8B3E00E9461150E94ED2485E032
:1027E000481A8827580A2296A2E8B3E00E94841566
:1027F00083ED11E00E94A01500916803003011F0F4
:102800000C940614E8EBFBE40E948A15009168031F
:10281000013011F00C941014A9EBB3E00E94841560
:10282000C098C19A84EF91E00E942716C09AC1987F
:102830000027A9EDB0E08C9186FB0EF401E041E0A9
:10284000041711F00C942A14A7EDB0E0ECE1FBE4BE
:102850000E94DB210027A9EDB0E08C9186FB0EF4ED
:1028600001E040E0041711F00C943C14A7EDB0E037
:10287000EAE1FEE40E94DB21A9EDB0E08C9186FB49
:10288000882780F9809580FBA9EDB0E08C9186F9CE
:102890008C938FE714E10E94A015A7EDB0E00E9491
:1028A000841580E08093DA00A8E4B3E088278C9355
:1028B00080E08093D4000C94F802F894FFCF0F923C
:1028C0001F922F923F924F925F927F92AF92BF9250
:1028D0000F931F932F933F934F935F936F937F9328
:1028E0008F939F93AF93BF93CF93DF93EF93FF9318
:1028F0008FB78F9380E08093D1008F918FBFFF912E
:10290000EF91DF91CF91BF91AF919F918F917F9187
:102910006F915F914F913F912F911F910F91BF90B8
:10292000AF907F905F904F903F902F901F900F90AF
:10293000189581E00E94361681E00E94361681E0EB
:10294000AA81BB818C930E946815A881B9818C9360
:1029500081E00E943616AC81BD818C91EE81FF81B1
:1029600001E00A93A981BA810E94F824A881B98163
:102970004C91AA81BB810C9104170FB681E0481AD3
:102980008827580A22960FBE11F40C94CB140C948D
:10299000A3140C94E314AA81BB818C918F5F8C9358
:1029A000AC81BD810E942225482FAA81BB810C9158
:1029B000041718F011F00C94DF140C94E1140C942B
:1029C000E3140C94A31482E0481A8827580A24962A
:1029D000089581E00E9436168BE00E943616A88189
:1029E000B98188278C930E946815AA81BB818C933A
:1029F000AA81BB818C91A881B9818F930E946115B6
:102A00008F918D9388278C938CE2482FAA81BB816C
:102A10000C91041711F00C94F314E881F9810AE089
:102A2000AC81BD810E94FF248CE0481A8827580A97
:102A300024960895F894FFCF481A8827580A0895D5
:102A4000480E8827581E089500FC10D0089503D022
:102A50001ED001F8F9CF0024E89457FF02C009D036
:102A6000689400F80BD010F80124089502D009D022
:102A70000895509540954F5F5F4F0895E89417FF74
:102A80000895009510950F5F1F4F68940895352F96
:102A9000242FE894452B11F468940895512F402F6A
:102AA0000027112780E1440F551F001F111F021B33
:102AB000130B416018F4020F131F4E7F8A9599F78C
:102AC00008958F938D918823E9F711978F91089539
:102AD0005F9BFECF8CB10895A0E6B7E08D9188236F
:102AE00011F00CD0FBCF08950E940723802D11F028
:102AF00005D0FACF08958DE001D08AE05D9BFECF2E
:102B00008CB90895A0E6B7E08D91882311F06CD0C0
:102B1000FBCF08950E940723802D11F065D0FACFD6
:102B2000089581E067D015D080E864C08FE7213038
:102B300039F08FEB223021F083E9233009F083ED67
:102B4000810F0C94FA1588EE93E081D03197D9F774
:102B5000089583E099277BC08AEF90E00E942716B2
:102B6000A39AA29AA19AA09AA59AA49AAC9885E051
:102B700090E00E942716AD98AB98AA98A99AA89AB7
:102B8000AD9AEF93FF93ECE8F1E00E941B16FF91E2
:102B9000EF91AD9859D0AD9AEF93FF93ECE8F1E047
:102BA0000E941B16FF91EF91AD984ED0AD9AEF9316
:102BB000FF93ECE8F1E00E941B16FF91EF91AD98B6
:102BC00043D0A898AD9AEF93FF93ECE8F1E00E9410
:102BD0001B16FF91EF91AD9837D088E20BD08EE0B5
:102BE00009D086E007D00895AC9A829505D004D02C
:102BF0002BD00895AC98F9CF859510F4A89A01C010
:102C0000A898859510F4A99A01C0A998859510F403
:102C1000AA9A01C0AA98859510F4AB9A01C0AB9806
:102C2000AD9AEF93FF93ECE8F1E00E941B16FF9141
:102C3000EF91AD9808953197F1F70895689462F88F
:102C40000895E89462F8089581E090E000C0EF9361
:102C5000FF93EE27E82BE92B31F0E0EAFFE0319714
:102C6000F1F70197D1F7FF91EF9108955A924A92A7
:102C7000480E8827581E08958DE207FD8D938F2DED
:102C8000881F802F881F8F57082F6894F7F8802F90
:102C900087FF15C080958395082F80E38D938EE282
:102CA0008D93802F815228F080E38D9399279C93F8
:102CB000089544270A95802F09F196D01FC08052AD
:102CC00030F09EE49D9381E48D939D93EFCF442754
:102CD000DF92EF92FF920F938FE1801B11F0082F8C
:102CE00083D089D09EE29D930F91FF90EF90DF906B
:102CF00044270395003209F4D7CF2BD03F93E8E85F
:102D0000FDE238E12F2D1E2D0D2DFF24EE24DD24B4
:102D10004427000F111F221FA8F42F923F920E94F8
:102D20000723102C0E940723202C0E940723302CFD
:102D30000E9407233197410DD21CE31CF01C3F90E9
:102D40002F9001C0339631963A9519F73F9107D0ED
:102D5000AFCFDD0CEE1CFF1C0A95D9F708950027B4
:102D600019E058D08F93802B11F0039501C08F91FB
:102D70001A95B9F7802F882309F496CF8F91805D3B
:102D80008D930A95D9F792CF0065CD1D80B2E60EDE
:102D900040597307A0ACB90350D6DC01286BEE0094
:102DA00094357700CA9A3B0065CD1D00B2E60E004F
:102DB00059730700ACB90300D6DC01006BEE0000CC
:102DC000357700009A3B0000CD1D0000E60E0000A4
:102DD00073070000B9030000DC010000EE000000F2
:102DE000770000003B000000F694E794D7944795E5
:102DF0000A95D1F7089500270DD08F9303958F2D55
:102E00008E298D29842BC1F78F91805D8D930A9532
:102E1000D9F74CCF1F930F93002710E2440FDD1C0E
:102E2000EE1CFF1C001F802F9AE0890B10F0082F6A
:102E300043951A9599F7802F0F911F9108958A93C2
:102E40000E948D1FFD0100D3888187F98883FA9342
:102E5000EA93E0E5F5E30E94471FA8F188E2A9D0D4
:102E6000FA93EA93AA85BB85E8ECF6E394E04ED3A7
:102E7000AA85BB85EC85FD850E94C71BAA85BB85FD
:102E8000FD010E94711CACE0BB27EA85FB850E9416
:102E9000C0209C2D97708E85890F8E87969520F483
:102EA000AA85BB850E94A91CA885B9850FD0AE81D3
:102EB000BF810CD0AC81BD8109D0EC85FD85C4D229
:102EC0002A960E94D5218A8123960895EA81FB8162
:102ED000E883F983EA85FB850E94C71BAA81BB8131
:102EE000EC85FD85E883F9830C94771BBA93AA934C
:102EF00085918A9385918A93FA93EA93BA93AA93D8
:102F000087FD09C0EC85FD85E883F983E885F985AF
:102F1000DF010E94C71B8C8180FD3CC0AE81BF8158
:102F2000EA81FB810E946E1FEA83FB838D818A9573
:102F30008D83AE81BF81A883B983AC85BD85E881CF
:102F4000F9810E94C71BEA81FB81AA85BB850E948B
:102F50006E1FEA83FB83E881F9810E948C1B8D81BF
:102F60008A958D8351F78C8181FD1DD08C8182FDE6
:102F70001AD08C8183FF03C0A885B98516D08C81B7
:102F800084FF06C0A885B985E881F9810E948C1B61
:102F900028960895AE81BF81A883B983EC85FD850D
:102FA0000E948D1FD0CFAC85BD85E881F9810C943E
:102FB000C71B8F930E94C8218F91885021F01896CB
:102FC000BA93AA93FACF08950E946B1C82E003C0C3
:102FD0000E946B1C80E48F930CE09DD28F9109F0CE
:102FE00008958F931ED28F9108F08BC28A93BA9363
:102FF000AA9325DF82FB839582F98A8388E1D9DF52
:10300000DF01EE81FF81FA93EA938A850DD281FD7B
:1030100006C008F434C0E2E9F5E352D218C0B0F1BA
:10302000E0E6F5E34DD2EC81FD811FD282F011D2B2
:10303000AE81BF81A883B9830E948C1BA885B98506
:1030400023D2A885B985EE81FF810E948C1BEE8179
:10305000FF810E94951F8A8531FD06C082FBFED14B
:1030600086FF02C087FDEBD1EE81FF81A885B9857F
:103070000E948D1F26960E94D52123960895E885EB
:10308000F985AE81BF810E948D1FE1CFAE81BF81E6
:10309000FBD1DDCF0E946B1C06E03DD209F0089504
:1030A000C3D108F40895D0D187F98A93BA93AA932B
:1030B000FFD140F019F02396FD011FC2A881B9810C
:1030C000EBD122C080E275DFE885F985FA93EA93B7
:1030D0001FE304EEACD1E8F4E4ECF5E3FFD1E6EF56
:1030E000F5E3F5D102D2E885F985AA85BB850E9472
:1030F000C71BEA85FB85E883F983A885B9850E940B
:103100008C1B28960E94D521E991F991899187FB22
:10311000A5C1AA81BB81B8D1AC81BD81A883B98387
:10312000EA81FB81AA85BB850E94771BE0E2F6E37A
:10313000D5D1EAE4F6E3CBD1D8D1EC81FD819DD1A4
:10314000DF0113D1AA81BB81AFD1AE81BF81A8833A
:10315000B983AC81BD81EA81FB810E94771BEC8140
:10316000FD81E883F983A885B9850E94C71BA885DE
:10317000B985ECE6F6E30E946E1FA885B985E88163
:10318000F9810E94771BEE81FF81E883F983AC818E
:10319000BD810E94771BEA85FB85E883F983EE8178
:1031A000FF81AA81BB810E948C1BABCF0E946B1C4C
:1031B0000CE0B1D109F0089555D187F98A93BA93FB
:1031C000AA9376D178F019F02396FD0196C18A81F1
:1031D000882322F0E881F98194D123C0A881B981A4
:1031E0005FD11FC00E94C721AA93BA938E8187FD29
:1031F00006C0EC81FD811FE300EE19D1A0F4EC8143
:10320000FD81DF0149DFAA81BB8146D1AC81BD814F
:10321000A883B983EA81FB810E94771B22960E94D2
:10322000D52123960895EC81FD81E883F9831DD192
:10323000AA81BB812DD1EA81FB81AC81BD810E9435
:10324000771BEC81FD81DF0190D0EC81FD81DF01F6
:1032500023DFEC81FD8111D1E1CF0E946B1C06E0E0
:103260005AD109F00895E0D008F40895EDD08827E8
:1032700087F98A93BA93AA9380E29BDEE885F98561
:10328000FA93EA931FE305EED2D080E048F110E410
:1032900003E0AC81BD81CBD0C8F4F6D0E885F985D8
:1032A000E883F983EA85FB850E948C1BEA85FB8510
:1032B000E883F983AC81BD810E94771BEA85FB8599
:1032C000A885B9850E94261C81E00AC0DDD0FD01D9
:1032D000B6D0AA85BB85A883B9830E94261C82E04C
:1032E0009C85982B9C87E4E7F6E3F8D0EEE9F6E3BB
:1032F000EED0FBD0E885F985AA85BB85A883B98384
:103300000E948C1B8C858F7719F1AE81BF81ECE612
:10331000F6E30E946E1F8C8580FF06C0EE81FF8160
:10332000A4D0E0E5F5E304C081FF02C0E8E5F5E3E1
:10333000AA81BB810E946E1FE881F981AE81BF81A5
:103340000E948C1BE881F981AA81BB810E948C1BA1
:103350008C8587FF03C0EA85FB8571D028960E9483
:10336000D521239608950E946B1C07E1D4D009F063
:103370000895BA93AA930E94BA1F80E11ADEFA93C5
:10338000EA9341505C4F40FB569547950695F7945C
:1033900003F98F2D902F93FF04C0809590958F5F38
:1033A0009F4F9F702ED02DD0006166270E941F2056
:1033B000EC81FD810E94751F83E08F93AA81BB8100
:1033C000A883B983EE81FF81AC81BD810E94261C58
:1033D000AC81BD81A883B983EA81FB810E948C1BEB
:1033E000EC81FD8142D08F918A9539F7EC81FD8186
:1033F000AE81BF810E948D1F24960E94D521229606
:10340000089533E0969587953A95E1F7F81A090BF8
:1034100008950E946B1C0E948D1FE8E4F5E30C9454
:10342000C91C0FEC11E403C006E41EE300C03681A2
:10343000301737810FB63F770FBE310708951781D8
:1034400030E8132717830895178117FB1F77178319
:103450000895178117FB106817830895178117F9CE
:1034600017830895178117FB08950681178100516E
:10347000104010F006831783089506811781005FBE
:103480001F4F068317830895E0E4F3E40C946E1F46
:10349000E8E4F3E40C946E1FE8E5F5E30C946E1F8A
:1034A000E0E4F5E30C946E1FE0E5F5E30C946E1F89
:1034B000E0E4F3E40E94471F8FB718978FBF089589
:1034C000A885B985A883B983AE81BF810FCDAA85B0
:1034D000BB85A883B983AE81BF8108CDAA85BB8592
:1034E000A883B983A885B98501CDE885F985E883E6
:1034F000F983AE81BF810C94261C0E9471200C942C
:10350000751F0E9466200C94751F18960E946E1FEE
:103510009A95D9F708950E948D1FFD010E94951F6D
:1035200004FF02C037FD09C003FF02C030FD05C023
:103530000770032319F4AC010895DFDF9894089510
:10354000182D4454FB210940399D52A246DF913F7A
:10355000182D4454FB21E93F182D4454FB21F93F19
:103560000606D43888BEE9FAA8BDC4B1B4BD9EEE43
:10357000213EAD529C804F7E92BE9015CB19A0018A
:10358000FA3E7751C1166CC156BF4C55555555552D
:10359000A53F061A7CD5CF5A3AD9E53DEB9C2B8A3C
:1035A000E6E55ABE7DFEB157E31DC73ED561C119A0
:1035B000A0012ABFA6F810111111813F4955555598
:1035C0005555C5BF0602D38AD40B9B6B713F165C61
:1035D0003E334143E3BFD92D8A174BC715407B903B
:1035E00027DE314330C0599277DA07903340D5AFA8
:1035F000CE066C6520C00581AB0E5E0B597B2DC0DD
:103600005490FE25C09F5140D776356DBB6562C092
:103610009DBFFF8456706140AC07360A229848C0AF
:103620000582089F8E98C34F683F0F29F95992076A
:10363000E2BF6A3EF3BAF5DF1B4068AB01ACAA916A
:1036400039C01D08F34062893C4004818C5DBFB6DF
:10365000A2F235C0427F6AAF19626240EE63909574
:1036600008FE77C0BE44B6B009677540075C1433E6
:1036700026A6913C050A9425F7A17F00ECBF7A802D
:103680006B5B542830C0730288368CC052C025BA98
:10369000052DBFB85EC08EEC28FD693650C005818F
:1036A0003C60145BC4DB384025FAB843DDA06440BD
:1036B0003BBEE2D2180E7B40EA49B0133F567E4033
:1036C000EC62BDFB9E51684083C8C96D305FF43F1A
:1036D00000000040FB21E93F000000002D44643E53
:1036E0007051CC989846E83CEBD404D010C40F013C
:1036F00001D010C4FD01FF93EF9387818F9390E871
:1037000089278783F0010BD08F91EF91FF918783F9
:103710000895D6D404D0FBC30F0101D0FBC300E051
:10372000E6D409F008959A01281B390B1AF4D00148
:103730000F01F5CF00272733300708F00BC5822F84
:1037400019D42DD43BD4372F36270AF45FD4F00197
:103750008081A80E8181B81E8281C81E8381D81EF7
:103760008481E81E8581F81E86818F708061081F24
:103770001AF44CD480E8682705FF02C081E01CD40D
:1037800004FD01C07FD434C49BD404D0C0C30F0156
:1037900001D0C0C308E1ABD409F00895480F591F08
:1037A0004F5F534067276F935F934F938FD42227C8
:1037B000F001EBD393E0110F331F441F551F661F19
:1037C000771F881F9A95B9F7FD01A7E0BB27919154
:1037D000A13011F49F709061992301F1939FA00C87
:1037E000B11CBB1F959FB695C01CD11CBB1F979FDA
:1037F000B695E01CF11C0B1F919F200DA11CBB1F57
:10380000949FB695B01CC11CBB1F969FB695D01C4B
:10381000E11CBB1F989FB695F01C011DAA9549F0AD
:103820002A2DAB2CBC2CCD2CDE2CEF2CF02E00271F
:10383000CECF4F915F916F9104FB16F0D0D302C0B1
:103840004F5F5F4FD5C33CD404D061C30F0101D09B
:1038500061C304E24CD409F00895481B590B415050
:103860005C4F67276F935F934F93F00183D32FEFE4
:10387000FD018BD3ADE3BA2FB77019F420952F93C8
:103880002FEFA116B306C406D506E606F70608070D
:1038900038F0A11AB30AC40AD50AE60AF70A080BD7
:1038A000221FAA0CBB1CCC1CDD1CEE1CFF1C001F25
:1038B000AA9509F72095AF90BF90CF90DF90EF9039
:1038C000FF900F914F915F916F9104FB1EF087D392
:1038D000415050408DC3E881F981AA81BB81089590
:1038E000FADF1BD3FD0121D3AC0199273F7711F5F6
:1038F0004F5F53401AF4EAD39FEFF7C25523D1F438
:103900004533C0F441954C5C9927483030F08081B4
:10391000982B882781934850F8CF7FEF80814423EC
:1039200019F0770F4A95FBCF672F60956823962B88
:10393000872380830895CFDF878187FFD2CFBF930E
:10394000AF93CFDFEF91FF91992311F0DF0104C016
:103950000895E0E4F3E403C0E0E4F3E40DC05D01A6
:10396000FF93EF9314D5EF91FF91B8D2F501FA933D
:10397000EA93D2DE229619C55D01FF93EF9307D536
:10398000EF91FF91ABD2F501FA93EA93B0DE229664
:103990000CC55D01FF93EF93FAD4EF91FF919ED296
:1039A000F501FA93EA93F3DE2296FFC4BA93AA9341
:1039B000FA93EA9388278A930A93229702D028964B
:1039C0000895B3D28C013323E9F0AE81BF8137FF74
:1039D00002C08DE28D9331FF05C080E38D9388276F
:1039E0008D93089530FF05C0E4E8F3E40E94DB21E5
:1039F000F6CF32FF05C0E0E8F3E40E94DB21EFCF11
:103A0000AE83BF8380E10E94C8212497AA83BB8331
:103A10003896E883F983EA85FB857FD2EC81FD81C6
:103A200087818F7787832FEF33E00217130738F5ED
:103A3000E2E0F3E487E099279B878A87AC81BD8128
:103A400026D29B8501F4991F9B8790FF0BC0B097EE
:103A5000B097A881B98142D2F896EE83FF8394DEB5
:103A6000EE81FF818A858A9541F7A881B981B09757
:103A7000B09734D289DE9B85939591951DC0EAEC71
:103A8000F2E487E09FEF9B878A87AC81BD81FFD1FD
:103A90009B85991F9B8790FD0AC0F096A881B981EC
:103AA0001DD2F897EE83FF836FDEEE81FF818A855A
:103AB0008A9551F79B8590959B878C859D858A83F8
:103AC0009B83EC81FD8131D2AC0154D211274D5F33
:103AD0005340483048F0102F0F2DFE2CED2CDC2CDD
:103AE000CB2CBA2CAA244850442351F0AA0CBB1C5E
:103AF000CC1CDD1CEE1CFF1C001F111F4A95F4CFCF
:103B0000AC85BD851196AC87BD87AA83BB83AFE822
:103B1000AF8330E8EAE3F2E43E83ABD2BFEFA4E048
:103B2000A216B306C406D506E606F7060807190767
:103B300040F0A21AB30AC40AD50AE60AF70A080B2B
:103B4000190BBB1F96958795779567955795479560
:103B50003795279548F40024201D301D401D501D29
:103B6000601D701D801D901DAA95D1F6B0952B2F5C
:103B700020633E814F8133231AF4203309F05FD054
:103B8000AC85BD852D93AC87BD873395431720F653
:103B90002FD014D08B85882371F095E49D931AF46F
:103BA00081959DE29D93982F880F890F9927991FE2
:103BB0008A879B8753D024960C94D521AA81BB81F8
:103BC000FD01119793E081919A9511F08033D9F31B
:103BD000939501C081918D939A95E1F78081882317
:103BE00009F08EE28D9388238191E1F71197089572
:103BF0009885992309F090E3882732508E932533D6
:103C000050F49923D9F432508E918033B9F49C93B7
:103C10003A95D1F708958E9183958A3311F08C935C
:103C200008959C933A95323009F490E33F3F99F719
:103C300081E312968C938B8583958B8708953F77CC
:103C40004885442311F04F3008F04EE04D5F532F6C
:103C5000515F451708F0452F4F830895EAE3F3E4D9
:103C6000689423E004E01FEF65917591861797072C
:103C700010F0861B970B111F769567950A95B1F783
:103C800010951EF4112319F0E89410631D932A95E2
:103C900049F711271C930895FA93EA93BA93AA93CC
:103CA00099279A939A939A939A93662700271127B4
:103CB00063958D91882391F1803219F4992311F540
:103CC000F7CF8D3221F49923E9F49068F1CF8E3249
:103CD00029F490FD17C068839160EACF782F7F7D2B
:103CE000753431F490FF68839A830E94BB2418C016
:103CF0008033F1F238F08A3328F491FDD9CF926005
:103D00006983D6CFEED103C0E8D101C0DFD19A815B
:103D100097FB17F92296FBD02696089590FF6883AB
:103D20009A8348815981552389F3451B1AF04A9596
:103D3000552701C05FEF040F151F42F42AEC3EEF38
:103D40000217130718F30250104005C025E331E0B5
:103D500020173107C8F243E055270E9427154883F2
:103D6000019547FF0E5F000F000F000F802FAED1AF
:103D7000AC81BD81EAE3F2E4E80F8827F81FAC814B
:103D8000BD8189818A95A80F8827B81F91E19B83FF
:103D900002C0AC81BD818D91AC83BD838E32D9F3DD
:103DA0009B819A9509F19B838033F0F08A33E0F48C
:103DB0008F7011F43896EFCFA82FA2955AD1AA0F81
:103DC00040F4A20EB31EC41ED51EE61EF71E081F29
:103DD000191FAA23F1F296958795779567955795C0
:103DE000479537952795EBCF4DEF53E022271032BB
:103DF00058F02A2DAB2CBC2CCD2CDE2CEF2CF02E29
:103E0000012F1127485F5F4F80E290E008171907E4
:103E100060F016950795F794E794D794C794B794F4
:103E2000A79427954F5F5F4FF1CF6A81E1D0EE8174
:103E3000FF815BD08881882331F188E00E94C8210E
:103E40008A81E883F983E885F985EA83FB83EC833B
:103E5000FD83880F20F48195E2E0F3E402C0EAECF0
:103E6000F2E4880F10F038960AC08F93A881B981C8
:103E700035D0FF93EF9388DCEF91FF918F918823EA
:103E800081F70E94D52128960895A881B9816617E7
:103E900078E06FB78D9195917A9599F06FBF89070A
:103EA0006FB7F8CFE881F981AA81BB81661778E006
:103EB0006FB78D9191917A9521F06FBF89076FB798
:103EC000F8CF70E8872797276FBF890731F06FB762
:103ED000892B12F071E067276FBF089588E0059085
:103EE0000D928A95E1F718970895A082B182C28257
:103EF000D382E482F582068317830895A080B1807F
:103F0000C280D380E480F580068117810895EC811A
:103F1000FD81EBCFE881F981E8CF88E091919D9315
:103F20008A95E1F718973897089586819781332706
:103F300097FB37F988949F7721F4882311F4326036
:103F400008952FEE28172FE7290740F42FE02823A4
:103F5000089411F43160089534600895807F969537
:103F60008795969587959695879596958795989434
:103F700088940895A080B180C280D380E480F580C9
:103F800006810F70006122270895108131814281DE
:103F900053816481758186818F7080610895883036
:103FA00050F02A2DAB2CBC2CCD2CDE2CEF2CF02E7F
:103FB00000278850F4CF0895689401C0E8948823BE
:103FC00069F00595F794E794D794C794B794A794AC
:103FD000279516F44F5F5F4F8A95F1CF0895220F12
:103FE000AA1CBB1CCC1CDD1CEE1CFF1C001F089572
:103FF00001D025C0203848F011F4A0FE06C0089476
:1040000012D005FF089581E0D7CF08952095A094A0
:10401000B094C094D094E094F09400950F92002452
:104020000894201D0F9050F40F920024A01CB01C87
:10403000C01CD01CE01CF01C001D0F9008955523DF
:10404000B2F0352F342B99F03FEF431737E0530789
:1040500078F4440F551F440F551F440F551F440F4C
:10406000551F0F7E042B152F67FB17F908952EC0DF
:1040700034C0259135914591559165917591859102
:104080009591089587E03F2D303230E0030778F4B2
:104090000F2DFE2CED2CDC2CCB2CBA2CA22E2227A3
:1040A000485050408A9579F7442755270FC088E03B
:1040B00004FD05C094DF415050408A95C9F708952A
:1040C000EA81FB81A881B9810F010895AA24BB244C
:1040D00065017501850198940895F8DF00EF1FE7E9
:1040E00008958FEFA82EB82EF3DF1F7708951DDFF8
:1040F000632FAC01FD0119DF732F00C0372F362B62
:104100003F7709F4089532FDECCF262F2727372F6C
:1041100060FB32F961FB33F93F70E0E5F3E4002323
:1041200011F427FD3C96030FE00F0027F01F849148
:1041300087FDD7CF86FDD1DF85FDC8DF84FD0AD09E
:1041400083FD0AD082FD0AD081FD0BD080FD0BD00B
:1041500098940895F001D2CEFD01D0CE67FB17F9F7
:10416000089577FBFCCF27FBFACFC094D094E0945E
:10417000F09481E0C80E8827D81EE81EF81E089526
:10418000D4DE31FD19C032FD17C030FD2AC08E5F6C
:10419000934092F0992329F5803238F4EBDE819533
:1041A0008B5DFDDEE8940ADF0CC0CC24C094DC2CCF
:1041B000EC2CFC2CF69412C0CC24DD24EE24FF243D
:1041C00010C080E8B81650F031F4BA28B22AB816F8
:1041D00011F4C0FC03C0CDDFF7FCE7CF37FF01C00F
:1041E000C4DFCD92DD92ED92FD9208956FDF0E94C3
:1041F0001B22602F6078FF0C001F0894F794402F5B
:10420000002311F463DF17C00F3F41F4FF2021F4B6
:1042100064DF67FB17F90FC064DF0DC011270027AB
:1042200085E0DD0CEE1CFF1C001F8A95D1F7552799
:1042300040585C4F04DFFD0158CE00000000000034
:1042400000C8000000000000001400000000000092
:10425000000233333333333333001F85EB51B81E41
:104260000500508D976E12830000228E75711B0D14
:104270000000378E588B4F0100006C41EF8D2100FC
:1042800000005853FE5A03000000893BE655000029
:104290000000F405970800000000FFE6DB000000C6
:1042A000000080FD150000000000F3320200000055
:1042B00000004C38000000000000A10500000000D4
:1042C00000009000000000000000EB24A7F11E0E8B
:1042D000CC6763B3D86275F6DD5373C8A1A031E52E
:1042E000E549B49DD9794378EA44000000A2941AC4
:1042F0006D420000000080842E410000000000405C
:104300008F407A84EA6EF03F1218AAAEFF5E8016E4
:10431000012CD82F768A4F62F735A78EA899C257FD
:10432000F33A11EA2D819997713D8DEDB5A0F7C64D
:10433000B03EFCA9F1D24D62503F2003500008006E
:10434000000000000000F03F000000000000E03F1F
:1043500000081000101010000808200000081000CD
:10436000108010000808200000412000414180001A
:104370002080200000204400418044002020800054
:104380004E414E00496E66696E697479000088E09E
:104390000FB6F8945A924A92E42DF52DA42DB52D1E
:1043A000480E8827581E0FBE08950FB6F8944990FE
:1043B00059900FBE08950E9407230D920020D9F74F
:1043C000089599910027A90FB01F1197492F4A9579
:1043D0005E2F6F2FE89411274395203019F0C89570
:1043E000802D01C080818823B9F07C917723A1F0D2
:1043F000781739F40EF0042F1395689411963196BE
:10440000EBCF112321F0411BA11B1127B10BE89425
:10441000E52FF62F1196E0CF882311F0002708959D
:104420000895D094E094F09491E0D90E9927E91E74
:10443000F91E10950895D190E190F19001910895A1
:1044400021913191419151910895102F90E8FF0CE5
:10445000001F0927990FF7941078652F90E8440FF3
:10446000551F5927990F4795607800380895FF0C1C
:1044700090E89027110F9795F794092F0895502FE2
:104480002D2D3E2D4F2D612F08952DEC3CEC4CEC45
:104490005DE366270FC0CFDFF2DFDD24EE2490E876
:1044A000F92E0FE307C0CCDF05C02227332740E2F7
:1044B00051E46627552351F1002381F1C6DF71F1E4
:1044C0001627005850580894050B18F407FD03C030
:1044D00025C007FD23C0469537952795F694E794A8
:1044E000D79422D0FF202AF0DD0CEE1CFF1C0150D7
:1044F00073F09D2D969548F0DD203AF4EE202AF4D5
:1045000091E0D90E9927E91EF91EB1CF07C09FE7A8
:10451000092FF92A9FEFD92EE92E0895DD24EE24E4
:10452000FF240027112708959F929924AA24BB24D1
:1045300088E1D216E306F40628F0D21AE30AF40A58
:10454000089401C08894991CAA1CBB1CDD0CEE1CAD
:10455000FF1C8A9571F7D92CEA2CFB2C9F900895AB
:104560000AF045D084CF5FE322273327442701C0D8
:1045700067DF6BDF5038B1F3003899F3902F951B4C
:104580008BF312F434D0FACF983118F02227332766
:104590004427983028F0232F342F44279850F9CF00
:1045A000992329F04695379527959A95D9F7912F14
:1045B000962742F014D0B0F6F794E794D7940F5FA3
:1045C0008BF6A5CF10D051F008F42BDFFF2052F26C
:1045D000DD0CEE1CFF1C0150CBF799CF9FCFD20E04
:1045E000E31EF41E0895D21AE30AF40A0895DF9236
:1045F000EF92FF920F931F93D22EE32EF42E052FEE
:10460000162F6F915F914F913F912F910895C8950B
:10461000319600200895FBDF202DF9DF302DF7DFE4
:10462000402DF5DF502D089507FB00680EF40F773D
:1046300057FB50680EF45F7707FD02C057FF05C0B7
:10464000D216E306F406050708952D153E054F051D
:10465000500708950E942116E89488278A938A9328
:104660005DDF11278D918032E9F31197BBD098F06F
:104670008D3229F4109511968C91B4D060F08E3261
:1046800029F411968C91AED008F446C022960E946F
:104690001E1681E008958C91A5D0D8F547D01196CB
:1046A000D0F703958D919ED0E0F38E3229F48C9152
:1046B00099D010F41196FBCF853419F0853609F0A6
:1046C00055C011968C918ED060F08D3219F08B32DE
:1046D00021F0DCCF08800094088211968C9182D062
:1046E000A8F68053898311968C917CD058F49981D7
:1046F000990F990F0980900D990F8053890F898325
:10470000873220F68981988199230AF48195080FD0
:104710002DC08E3289F611968C9164D068F606D041
:1047200018F011960A95F8CF1196C1CF4F2D3E2D56
:104730002D2DDD0CEE1CFF1CA8F0DD0CEE1CFF1C6B
:1047400088F0D20EE31EF41E68F0DD0CEE1CFF1C98
:1047500048F0805309F06894D80E8827E81EF81EA8
:1047600008F00895F42EE32ED22E089534D019F1D6
:1047700016F5098308E921D00695882787959F2D8E
:104780009F77980FF92E0150000F110F079589811F
:10479000882379F01AF48195898306C076DE8981B1
:1047A0008A958983D9F705C080DE89818A958983B6
:1047B000D9F722960895B2DEFCCF0DD041F0FF204C
:1047C00032F00A9531F0DD0CEE1CFF1CD2F7889414
:1047D00008950894089500240D280E280F28002A13
:1047E00000200895803320F08A3310F4089408954F
:1047F0008894089599278D9193958823E1F793954F
:1048000011968C9311978E919A95D1F70895EA2F6E
:10481000FB2F00244C918D9103948E32E1F71124EB
:104820008D9113948823E1F71A94101640F4119790
:10483000202F2119239580E38D932A95E9F71130D4
:1048400039F59927AE2FBF2FA00DB91FA00FB91FA3
:104850008C919C93853308F421C031E08E918E3287
:10486000E9F38D3241F0830F8A3319F480E331E0AC
:1048700001C033278C93AE1789F7332341F0AE2F55
:10488000BF2FB8DF81E34D3209F43196808308955C
:104890008827E00DF81FE00FF81F80830895040FAC
:1048A000151F261F371F0895000F111F221F331FCA
:1048B000089500951095209530950F5F1F4F2F4F4D
:1048C0003F4F0895019110810EC0019111912191E6
:1048D00030810BC00191108117FF05C03FEF2FEF12
:1048E00004C0008111272227332737FF03C0E1DFEF
:1048F0008DE28D93CF93DF93CF92DF92EF92AA2434
:10490000BB24CC24DD24EE2440E2CAE0DD2755E0C0
:1049100093E38881890F87FD9F7083FD907F891BBA
:1049200089935A95A9F7C0DFAA1CBB1CCC1CDD1CBF
:10493000EE1C4A9551F7E894EFE0FF2782910ED0E4
:10494000EB30E0F71EF068948A2D0CD088278D9309
:10495000EF90DF90CF90DF91CF910895982F8295BF
:1049600001D0892F8F70805D26F0803309F408957F
:1049700068948D93089500271127222733271DD08F
:104980008A3328F4803318F005D015D0F9CF0EF40F
:1049900090CF089580538F93402F512F622F732F04
:1049A00083DF82DF7CDF80DF8F919927080F191F5B
:1049B000291F391F08958D910895E894FCDF8032F6
:1049C000E9F38B32D9F38930C9F38D3211F468944D
:1049D000F2CF089588278D93089581918D93882330
:1049E000E1F7089594E081918D939A95E1F7089508
:1049F00009919191992351F08A95D9F73197819135
:104A00008D930A9519F08823D1F70895E3CFE199A2
:104A1000FECFEEBBFFBB31960895F9DF8D917B375A
:104A200029F48DBBE29AE19A8823B9F77727089594
:104A300091E001C092E0EBDFE09A8DB38D939A95FF
:104A4000D1F708958FEF83959D919923E1F708950C
:104A5000689401C0E894AF93BF938D9116F0919143
:104A600003C00E940723902D891718F011F48823A2
:104A7000A1F7BF91AF91089550455254FB210940D1
:104A80001DE1639946DF913F000070420080BB4505
:104A900000606A47C976BE9F3AE3B8404C37894107
:104AA00060E0AA40000000000000F03F00000000AD
:104AB00000000040000000000000000000000000B6
:104AC00000807640000000000060564000000000BA
:104AD00000A056400000000000805640000000008A
:104AE000007066400000000000906640000000007A
:104AF000008066400000000000D870400000000008
:104B000000E870400000000000E07040000000007D
:104B1000007876400000803F0000C8422D00202031
:104B20002057504C5452414B2020563662202020B2
:104B3000202000002D2D2D2D2D2D2D2D2D2D2D2D19
:104B40002D2D2D2D2D2D2D2D000020202020284312
:104B50002932303039204B484820202020200000C6
:104B600020646A376F6F40742D6F6E6C696E652EAE
:104B700064652020000020434F4E4649475552416E
:104B800054494F4E204D4F4445200000204C415485
:104B90002E203A20202020202020202020202020ED
:104BA0000000204C4F4E2E203A2020202020202094
:104BB0002020202020200000202020202020202035
:104BC00020202020202020202020202000004B6FAB
:104BD0006E66696775726174696F6E732D4D6F646F
:104BE000757300004765626520456967656E706F83
:104BF000736974696F6E204272656974656E67725D
:104C0000616420696D20466F726D61742047472E84
:104C100047474747472065696E2000004265656E3B
:104C200064652045696E67616265206D6974204323
:104C3000686172616B746572203A20232000230042
:104C40004B6F6E74726F6C6C6175736C6573756E9F
:104C5000672061757320454550524F4D3A20000042
:104C60004765626520456967656E706F7369746931
:104C70006F6E204C61656E67656E67726164206956
:104C80006D20466F726D6174204747472E47474736
:104C900047472065696E20006265656E6465204542
:104CA000696E67616265206D697420436861726135
:104CB0006B7465723A20230041627363686C75738C
:104CC0007320646573204B6F6E66696775726174DB
:104CD000696F6E732D4D6F6475733A00D666666E9C
:104CE00065204D617373656B6F6E74616B742076B4
:104CF0006F6E20506F72742050413020756E6420AA
:104D00007374617274652050726F6772616D6D208B
:104D10006E6575002043414C4C203A202020202015
:104D2000202020202020202000004765626520529E
:104D300065666572656E7A2D43616C6C202820670C
:104D400067662E20696E636C2E20535349442029D8
:104D50002065696E2000202057414954494E472064
:104D6000464F5220444154412020000047505750A4
:104D70004C2C00002A00300053005700DF002E00AA
:104D80002000244750524D432C00303000006B006F
:104D90004B006D004D00245047564F492C002C000D
:104DA0002C442C0045004E004750532046495820C3
:104DB000444154413A0041435455414C20475053DB
:104DC00020444154413A00004C41543A20202020D4
:104DD00000004C4F4E3A20202020000053454C4507
:104DE00043543A200000524543454956454420412A
:104DF0005052530046524F4D3A200000504F5349F5
:104E000054494F4E3A00494E43414C4C3A20000021
:0C4E10006973200020696E2000002B0058
:00000001FF
